:020000040000FA
:10000000C0310020AD020000B5020000B7020000C0
:10001000B9020000BB020000BD02000000000000A9
:1000200000000000000000000000000015020000B9
:10003000C10200000000000051020000C5020000E3
:10004000A1040000C7020000C7020000C7020000B0
:10005000C7020000C70200003D030000C702000005
:10006000C7020000C7020000C7020000C70200006C
:10007000C7020000C7020000C7020000C70200005C
:10008000C7020000F9040000C7020000C702000018
:10009000C7020000C7020000C7020000C70200003C
:1000A000C7020000C7020000C7020000C70200002C
:1000B000C7020000C70200000000000000000000AE
:1000C000C7020000C7020000C7020000C70200000C
:1000D000C7020000C7020000C702000000000000C5
:1000E0000000000000000000000000000000000010
:1000F0000000000000000000000000000000000000
:1001000000000000000000000000000000000000EF
:1001100000000000000000000000000000000000DF
:1001200000000000000000000000000000000000CF
:1001300000000000000000000000000000000000BF
:1001400000000000000000000000000000000000AF
:10015000000000000000000000000000000000009F
:10016000000000000000000000000000000000008F
:10017000000000000000000000000000000000007F
:10018000000000000000000000000000000000006F
:10019000000000000000000000000000000000005F
:1001A000000000000000000000000000000000004F
:1001B000000000000000000000000000000000003F
:1001C000000000000000000000000000000000002F
:1001D000000000000000000000000000000000001F
:1001E000000000000000000000000000000000000F
:1001F00000000000000000000000000000000000FF
:10020000DFF80CD000F088F8004800475D0A0000D5
:10021000C0310020244B19680868B0E8F04F80F323
:100220000988BFF36F8F4FF0000080F3118870478B
:10023000000000000548006880F3088862B661B6D7
:10024000BFF34F8FBFF36F8F00DF0000000000008F
:10025000EFF30980BFF36F8F134B1A681EF0100F76
:1002600008BF20ED108A20E9F04F106008B44FF06D
:10027000400080F31188BFF34F8FBFF36F8F01F001
:100280001FFA4FF0000080F3118808BC1968086855
:10029000B0E8F04F1EF0100F08BFB0EC108A80F3EA
:1002A0000988BFF36F8F704714000020064880470D
:1002B00006480047FEE7FEE7FEE7FEE7FEE7FEE74B
:1002C000FEE7FEE7FEE7FEE7610500000102000031
:1002D00040EA01039B0703D009E008C9121F08C0C8
:1002E000042AFAD203E011F8013B00F8013B521E48
:1002F000F9D27047D2B201E000F8012B491EFBD2BF
:1003000070470022F6E710B513460A460446194620
:10031000FFF7F0FF204610BD064C074D06E0E068F1
:1003200040F0010394E8070098471034AC42F6D33C
:10033000FFF76AFF281E0000481E00002DE9F04765
:1003400000268AB0DFF85091B0464FF48075012442
:1003500037460696284600F06FFC38B1D9F80403FA
:10036000204203D0284600F05DFC26432D1D64008A
:100370007F1CADB2082FEDD34FF4BE74204600F0C1
:100380005BFC48B1204600F04DFC46F0004606AA52
:100390000121002000F032FC404D16F0FF0F15D077
:1003A0000127002437420DD009EB8401D1F8100554
:1003B000D1F81015C0F3042055F82420C1F30141F1
:1003C00002B190477F00641C082CEBD3002E5FDA4B
:1003D0004FF0FF30CDF8108054E0281910F8507F0E
:1003E00090F9000027F0C008401C3BD007A9404608
:1003F00000F076FB10B34FEA9719404600F0D6FAAA
:1004000055F820701FB1B9F1030F03D006E0B9F120
:10041000030F27D104A9404600F06AFB4FF0A0412A
:1004200001EB8800D0F8000706A9C0F3014A404656
:1004300000F056FB18B1BAF1020F03D012E0BAF186
:10044000030F0FD1B9F1030F08D1BAF1020F1DD07C
:100450000221404600F0B6FB761CF6B217B14946C1
:100460004046B847641C042CB7D3002E10D06A460F
:100470000121002000F0C2FB06990098884207D0B5
:1004800006900498002634460790A6E70321E0E78B
:100490000AB0BDE8F0870000006000406011002055
:1004A00070B54FF48076304600F02CFB114CB5054A
:1004B00060B1304600F02DFB0120C5F808036079DB
:1004C00020B9012060712168002088474FF48276AE
:1004D000304600F017FB00280AD0304600F019FB28
:1004E0000220C5F808032168BDE8704001200847D4
:1004F00070BD0000640000202DE9F041164E4FF45D
:10050000A071304600F0A0FB0025EFF311844020DD
:1005100080F31188D6F804758100304600F094FB12
:1005200001F0FAFA381A20F07F46012E07D901F0BF
:10053000E5FA022803D0002601F0F4FA0543761EFE
:10054000FAD225B105494FF08050086040BFE0B2B3
:1005500080F31188BDE8F0810010014004ED00E057
:10056000F0B5B5480023021D0178101D01254FF09C
:10057000805406290BD11678360708D10678C6F3C1
:100580000316032E06D0042E04D0052E02D0062911
:1005900007D00EE0B4F82463A84FC6F304263E60EB
:1005A00002E01678360704D10678C6F30316032E48
:1005B00002D0062904D00FE0A24FA14E7E670EE0C4
:1005C0001678360708D10678C6F30316032E06D030
:1005D000042E04D0052E02D0062907D00EE0D4F850
:1005E0004462994FC6F342363E6002E01678360701
:1005F00004D10678C6F30316032E02D0062906D0CE
:1006000011E0924E376827F0807737600EE0167859
:10061000360708D10678C6F30316032E06D0042E3B
:1006200004D0052E02D006290AD011E04FF08046F2
:10063000C6F80C31C6F81031834E361F336002E025
:100640001678360704D10678C6F30316032E02D0B7
:10065000062905D00CE07C4F032664373E600AE093
:100660001678360704D10678C6F30316032E02D097
:1006700006290DD014E0764F05263E60744E78367C
:100680003560734E083633603F263F1D3E6002E002
:100690001678360704D10678C6F30316052E02D065
:1006A000062957D062E06B4E36686B4F3E60694E4C
:1006B000361D36683F1D3E60664E083636683F1D63
:1006C0003E60644E0C3636683F1D3E60614E10360B
:1006D00036683F1D3E605F4E143636683F1D3E60F3
:1006E0005C4E183636685C4F20373E60594E1C36DB
:1006F00036683F1D3E60574E203636683F1D3E60CF
:10070000544E243636683F1D3E60524E28363668B9
:100710003F1D3E604F4E2C3636683F1D3E604D4EAD
:10072000303636684C4F40373E604A4E3436366875
:100730003F1D3E60474E383636683F1D3E60454E91
:100740003C3636683F1D3E60424E403636683F1D9F
:100750003E6002E01678360708D10678C6F3031625
:10076000032E06D0042E04D0052E02D0062907D071
:1007700019E0D4F85812394A01F04F01116002E033
:10078000117809070FD10078C0F30310032803D0B4
:10079000042801D0052806D131480168C90702D0D4
:1007A0006FF001010160D4F83001062808D1D4F8B7
:1007B0003401062804D12B48016841F480610160AE
:1007C00022487438016841F470010160BFF34F8F13
:1007D000BFF36F8F4FF01021D1F80002002803DB28
:1007E000D1F80402002822DA1F4A15601F48046865
:1007F000002CFCD01524C1F800420568002DFCD067
:10080000C1F8044201680029FCD013600168002986
:10081000FCD0BFF34F8F0D48F0380168144A01F443
:10082000E06111430160BFF34F8F00BFFDE7124944
:1008300010480860F0BD0000E00F00F040350140B6
:100840000DF0ADBA00C007403C050040FCED00E0F3
:10085000105600400404001020C50040E40E004083
:10086000000400403C17004004E5014000E4014062
:100870000400FA050090D0037000002002E008C8D0
:10088000121F08C1002AFAD170477047002001E00A
:1008900001C1121F002AFBD17047000072B609483F
:1008A0000068C00700D000BEBFF34F8F0548E43892
:1008B0000168054A01F4E06111430160BFF34F8F05
:1008C00000BFFDE7F0ED00E00400FA050EB50021E1
:1008D0000091CDE901106A4644F20100FFF7DEFF06
:1008E0000EBD00F003B800F009B8000072B602486F
:1008F0000168491C016070476C00002003490868CA
:10090000401E086000D162B6704700006C000020F5
:100910002DE9FC410646C0074FF000050ED0104FF0
:1009200000240122385D009500231146019500F056
:1009300037F9641C042CF4D300F02EF8B0070DD561
:10094000074E0024361D0022305D0323009511461A
:10095000019500F025F9641C042CF4D3BDE8FC815A
:10096000181E000007490B5C4FF0A041D1F8042588
:100970000120984020EA0203C1F808351040C1F870
:100980000C057047181E00000249085C012100F0A8
:100990002AB90000181E000010B500242046FFF7F9
:1009A000F3FF641C042CF9D310BD00000249084475
:1009B00090F93000704700006011002070B5084CBD
:1009C000050009D010342168002907D0086820608C
:1009D000496828468847F6E70834F4E770BD000008
:1009E0004C110020054A012120B1012805D1917048
:1009F000FFF7E4BF51700020FAE770474C11002068
:100A000009490120096809B1002070470749CA69EE
:100A1000002AF9D1044A283212688968491E8A429C
:100A2000F3D1022070470000E810002014000020DD
:100A30000268134602E08A4204D01268002AFAD102
:100A40000B60016070470020FFF78CFFC82000F0AA
:100A5000B3FDF8E70120FFF785BF00001CB500F0EB
:100A600061F808B1FFF732FF0120FFF751FF144989
:100A70000220CDE9000100234FF4827211A1134836
:100A800001F010F812480090002301224FF47A710F
:100A900010A001F05FF90A4C606001F03DF80246D9
:100AA0000020034600900121606801F08DF90B4899
:100AB000016841F00401016000F0CAFDFEE700009A
:100AC000000000204C45443000000000470A0000B0
:100AD000550A00004C4544310000000010ED00E0D4
:100AE000C20800F007030120895C98400840704765
:100AF00010B5C20800F00703885C01249C40204325
:100B0000885410BD00F180400068002800D001200A
:100B1000704708B500F18040002101600068009036
:100B200008BD000070B50A4C207808B185250CE09E
:100B30000020A06060602061E060064800F0A0F83E
:100B4000054600F087F801202070284670BD00009F
:100B50004C110020E509000070B5104D0446A8783E
:100B600038B114B16168012088470020FFF7B9FE51
:100B70000CE00020FFF7B5FE24B1084821461030F4
:100B8000FFF756FFE86808B900F08AF8E868401CEB
:100B9000E860BDE870400020FFF7A5BE4C110020C2
:100BA00070B541EA4201DDE904564FF0A04441EA44
:100BB000830141EA052104EB800041EA0641C0F8C7
:100BC000001770BD4FF0A04202EB8000D0F8002764
:100BD00022F44032C0F80027D0F8002742EA014151
:100BE000C0F80017704701224FF0A043824011B1B6
:100BF000C3F808257047C3F80C25704718B5084B93
:100C00006C4601441B68009306E000BF54F8203096
:100C1000D3F81035401C08C28142F7D818BD000037
:100C2000241E0000034908B5084400210160006843
:100C3000009008BD0060004002494058012800D0E3
:100C4000002070470060004008B500224250405824
:100C5000009008BD08480068012110F0010F08D17C
:100C60004FF0E020E02280F80024C0F88012C0F8A5
:100C7000001102480160704700E100E018050040E3
:100C80000649024600200B790BB1852070470A60A7
:100C900001220A7100224A7170470000640000209E
:100CA00070B54FF48270FFF734FF02204107C1F89E
:100CB00004030B4B196841F0807018600948026802
:100CC00042F00104046044684FF40A554668361B3C
:100CD000AE42FBD30260196003490120086070BD79
:100CE000FCED00E0001000E0080000402DE9F041BC
:100CF000184C0F460546E6682068001D00F05AFBB8
:100D000038B9206890F82C1001208840216981436F
:100D10002161681C07D137B12168BDE8F0410E4858
:100D2000091D00F080BB20683544B542456021684C
:100D300005D2A06BBDE8F041091D00F05CBB606B03
:100D4000091D00F058FBA06A854200D2A562BDE8EB
:100D5000F081000014000020101100202DE9F04166
:100D6000054600F06DFB2E4CA068401CA06020687A
:100D70002C4F10B1606940B32DE02560A0680128B8
:100D800029D1002606EB860007EB800000F025FB4A
:100D9000761C032EF6D323483C3000F01EFB21487E
:100DA000503000F01AFB1F48643000F016FB1D485D
:100DB000783000F012FB1B488C3000F00EFB194815
:100DC0003C3060631430A06305E02068E96AC06AC3
:100DD000884200D82560606A401C6062E96A012090
:100DE000226988401043206101EB810007EB8000FD
:100DF000291D00F018FB00F02DFB606900280DD0C4
:100E00002068E96AC06A884208D207494FF08050DA
:100E1000086040BFBFF34F8FBFF36F8FBDE8F08115
:100E2000140000208410002004ED00E010B500F054
:100E300007FB0E4C2068A0B90D4800F0CEFA0C4814
:100E4000143000F0CAFA0A48E06014302061002231
:100E50001021202000F07CFC206010B105A100F0E2
:100E600075FBBDE8104000F0F5BA0000500000200E
:100E700024110020546D72510000000030B4026C47
:100E80000B46002A0BD0C1681144C1604468A142DE
:100E900001D30168C16030BC1846FFF719BA30BCF5
:100EA00070472DE9F041856B174604460026026C19
:100EB00082B1C7B1E068FFF70BFAE168206C091A4C
:100EC000E1602268914202D26168081AE060022F54
:100ED00016D017E02068A8B9606800F073FE0646D7
:100EE000002060600EE0A068FFF7F2F9216CA068B6
:100EF0000844A0606168884204D32068A06001E0D3
:100F000005B16D1E6D1CA5633046BDE8F08110B5BE
:100F10000446006B00F0A8FA2046BDE8104000F03F
:100F2000A3BA00000A4800210269012A00D9012160
:100F30000268D26A0AB100207047064A1268012A84
:100F4000F9D80029F7D1816AC068081A70470000F3
:100F500014000020841000201A4C1B4E12E000BF29
:100F600000F06EFAF068C568281D00F023FAA0684A
:100F7000401EA0606068401E606000F06BFA28466A
:100F8000FFF7C5FF60680028EAD10F48783800688D
:100F9000012808D90D494FF08050086040BFBFF3C9
:100FA0004F8FBFF36F8FFFF7BDFF0228D5D300F03F
:100FB0007FFBFFF7B7FF022801D300F077FA00F0BC
:100FC0006FFECAE714000020FC10002004ED00E0D2
:100FD0002DE9F0470E46DDE9098417468246910067
:100FE0009946089DA522206BFFF784F96FF0030155
:100FF000206B01EB8701084420F00707002022182E
:10100000315C82F83410315C11B1401C0428F6D3F5
:10101000002684F83760032D00D30225E562C4E979
:101020000E56201D00F0E4F904F1180000F0E0F97C
:101030002461C5F103006462A061266484F8446001
:101040004A465146384600F099F92060B8F1000F41
:1010500001D0C8F80040BDE8F087000070B500245A
:1010600041600B4D0061914206D8D11A82699142CC
:1010700006D2011D286907E09A4203D2994201D3A2
:10108000012403E0011DE86800F0B5F9204670BDB9
:101090005000002010B5044600F0D2F9A06B28B132
:1010A0005FF0000400F0D6F9204610BD0124F9E7F6
:1010B00030B589B0264D41E00498002806DADDE914
:1010C0000601059A90470498002837DB069C606962
:1010D00010B1201D00F06EF902A800F09DF8024644
:1010E00004980A282AD2DFE800F0050505291E2603
:1010F0000505291E0598A169034601442046FFF70E
:10110000ADFFD8B1616A20468847E069012815D152
:10111000002000900598A169002342181946204636
:1011200000F052FE0AE00598A0618118134620469F
:10113000FFF794FF02E0204600F096F9002204A990
:10114000286800F00DFC0028B6D109B030BD0000C1
:10115000500000202DE9FC410F46054600F0A8FA9A
:1011600001A800F059F80446019818B100F098FD64
:10117000BDE8FC811E4EB7B130690068A8B30027F6
:10118000291B3A46306800F0F5F900F089FD002887
:10119000EED118494FF08050086040BFBFF34F8F29
:1011A000BFF36F8FE4E7A542EAD800F079FDF0685D
:1011B0002746C068C468201D00F0FCF8E0690128DB
:1011C0000FD1A0692B4641193A462046FFF746FF4A
:1011D00038B100200346014600902A46204600F020
:1011E000F3FD616A20468847C2E7FFE70127C7E7AA
:1011F0005000002004ED00E00648416B096829B169
:10120000416BC968C9684968816270474FF0FF3116
:10121000FAE700001400002070B5054600F07CFCE1
:10122000064E0446B068844203D200F009F801205B
:1012300000E0002028602046B46070BD500000200F
:10124000F8B5144D1EE0C068C4680668201D00F0A3
:10125000B1F8616A20468847E069012812D1A06987
:101260003044B04206D924616060211DE86800F076
:10127000C2F807E0002003460146009032462046AF
:1012800000F0A2FDE86801680029DCD12969C5E900
:101290000310F8BD50000020402080F31188FEE7C5
:1012A000074CE068016841B1C0680021D0F8000037
:1012B000FFF750FFFFF7FCFEF3E701210020F7E7FF
:1012C000500000202DE9F041044600F0B9F894F9EF
:1012D000455004F1240609E0606A48B1304600F048
:1012E000A9FC08B100F08AF96D1E6DB2002DF3DC87
:1012F0004FF0FF3684F8456000F0ACF800F0A0F83D
:1013000094F9445004F1100709E0206948B13846C7
:1013100000F090FC08B100F071F96D1E6DB2002D67
:10132000F3DC84F84460BDE8F04100F093B80000BD
:1013300070B504460025400704D004F00700C0F152
:101340000800044400F0B4F90A49486818B90A488A
:1013500020F0070048600A6840F6F87310199842B8
:1013600004D2904202D94B6808609D1800F098FCA6
:10137000284670BD080000207C00002010B5084CF5
:10138000031F24681C601B1F1960191F054B0B608D
:1013900014390A60091F6FF0020244380A6010BD58
:1013A000201E000099120000EFF31180402181F30C
:1013B00011887047D0E9013201699A60D0E90123B0
:1013C0005A604A68824201D182684A600022026102
:1013D0000868401E08600868704700F108014FF077
:1013E000FF32C0E90112C160016100210160704754
:1013F00000210161704730B50B685A1C02D000F122
:10140000080202E0026904E02246546825689D4211
:10141000FAD953684B6099608A605160086101682D
:10142000491C016030BD42684A6093688B609368D4
:101430005960916008610168491C016070470000B3
:10144000402080F3118802480168491C0160704700
:101450001000002003490868401E086001D180F395
:1014600011887047100000207047000010B5002060
:10147000FFF772FB0B481F21C0F808150121C0F8C7
:101480000413816001600221C0F844130649E02082
:1014900081F800044FF0E0214FF40030C1F8000162
:1014A00010BD00000010014011E000E02DE9F04106
:1014B00004462448844200D9044672B6224DD5F829
:1014C0000475FFF79DFAD0B33819012120F07F4051
:1014D000C5F80813C5F840054FF4A07841462846E2
:1014E000FFF7B2FB4FF48030C5F80403BFF34F8F12
:1014F0004FF0E02634B120BFD6F80012D6F804220F
:101500001143F8D0C5F8080341462846FFF79CFB75
:101510004FF480712846FFF797FB0120C5F80403BC
:10152000D5F804054FF40031C01B20F07F40C6F809
:101530008012A04200D9204608B100F0B1F862B68E
:10154000BDE8F081FDFFFF000010014010B5084B21
:10155000002200BF53F832401CB1521C022AF9D3BA
:1015600010BD43F8321003EBC201486010BD00000B
:101570007410002070B515460E460446FFF760FF54
:1015800094F944100020491C01D184F8440094F9D6
:101590004510491C01D184F84500FFF75BFFA06BA3
:1015A00028B92A46314604F1240000F03DF82046CF
:1015B000BDE87040FFF786BE10B5020009D000F00C
:1015C00077F800211046FFF791FB00F069FB002837
:1015D00008D105494FF08050086040BFBFF34F8FDE
:1015E000BFF36F8F10BD000004ED00E002490A6AEE
:1015F0000260C96841607047140000200149012061
:10160000C86170471400002010B50C4605490968F0
:101610001831FFF7F0FE2046BDE810400121FFF72A
:1016200065BB00001400002070B50D460749144644
:1016300009681831FFF7F7FE0CB14FF0FF3521466E
:101640002846BDE87040FFF751BB000014000020A1
:101650001CB50F480024CDE9004023463C220DA1D3
:101660000E4800F01FFA012811D100F08FFB01286D
:101670000DD1402080F311880548611E2C3881620D
:1016800001214161C460BDE81C4000F03BB81CBDB5
:101690004000002049444C4500000000590F000064
:1016A0000249CA681044C860704700001400002056
:1016B0000248016B491C01637047000014000020C0
:1016C0000E48016B11B10121C16170470021C16158
:1016D00001690B4AB1FA81F1C1F11F0101EB8101EE
:1016E00002EB810101F108034A6852684A609A429C
:1016F00001D152684A60D16801607047140000202F
:10170000841000200E49E02081F8140DFFF7AEFE92
:101710000C49002008600C48016841F47001016028
:101720000A48016841F04041016007487838016883
:1017300041F010010160FEF77DFDFFF7ADFD0000F7
:101740000EE000E01000002088ED00E034EF00E043
:1017500070B50E00054612D005FB06F04830FFF7C5
:10176000E7FD040009D004F1480120464EB10160B4
:10177000C0E90F56012100F007F8204670BD002097
:10178000ECE70060F4E7000070B50D460446FFF793
:1017900057FED4E90F12206801FB020060600020B0
:1017A000A0632068A0600146E06B401E00FB0210B1
:1017B000E0604FF0FF3084F8440084F8450004F105
:1017C00010004DB1FFF709FE04F12400FFF705FEFC
:1017D000FFF740FE012070BD21690029F8D000F01C
:1017E00029FA0028F4D005494FF08050086040BF26
:1017F000BFF34F8FBFF36F8FEAE7000004ED00E007
:101800002DE9FF4700273C4E82B099468A460446A0
:10181000B8464FF0805500BFFFF712FEA06BE16B9A
:10182000884206D3B9F1020F03D00498C8B1DFB1E2
:101830001EE04A4651462046FFF733FB616A19B164
:1018400004F1240000F0F6F928B1356040BFBFF381
:101850004F8FBFF36F8FFFF7FDFD012006B0BDE88E
:10186000F087FFF7F7FD21E06846FFF7BFFE01278D
:10187000FFF7F0FDFFF71CFFFFF7E2FD94F94400CE
:10188000401C01D184F8448094F94500401C01D1EA
:1018900084F84580FFF7DEFD04A9684600F0DAF819
:1018A00030B12046FFF70EFD00F0FAF90020D5E731
:1018B000FFF7C6FDA06BE16B884214D1FFF7CAFDAC
:1018C00004F110000499FFF79FFE2046FFF7FAFC91
:1018D00000F0E6F900289FD1356040BFBFF34F8F7D
:1018E000BFF36F8F98E7FFF7B5FD2046FFF7EAFCDF
:1018F00000F0D6F990E7000004ED00E02DE9F04794
:101900009846174689460446FFF74EFDA16B0646EA
:10191000E06B814208D3B8F1020F05D00020F1B28C
:1019200081F31188BDE8F08794F945504246494655
:101930002046FFF7B6FA681C04D06D1C84F84550A9
:101940000120ECE7606A0028FAD004F1240000F0DE
:1019500071F90028F4D0002FF2D001203860EFE7B1
:101960002DE9F7470026DFF8E88083B08A46044671
:10197000B1464FF0805700BFFFF762FDA56BCDB1B8
:1019800051462046FFF77AFA6D1EA563206958B1CB
:1019900004F1100000F04EF930B1C8F8007040BFFB
:1019A000BFF34F8FBFF36F8FFFF754FD012006B0D9
:1019B000BDE8F087059808B11EB106E0FFF74AFDC3
:1019C00027E06846FFF712FE0126FFF743FDFFF709
:1019D0006FFEFFF735FD94F94400401C01D184F8F7
:1019E000449094F94500401C01D184F84590FFF7DC
:1019F00031FD05A9684600F02DF8002820460AD0E0
:101A0000FFF760FC00F04CF92046FFF743FB00288D
:101A1000B2D00020CBE7FFF73DFB98B104F12400E2
:101A20000599FFF7F1FD2046FFF74CFC00F038F96F
:101A30000028A1D1C8F8007040BFBFF34F8FBFF39B
:101A40006F8F99E72046FFF73DFC00F029F993E7F7
:101A500004ED00E02DE9F0410C460546FFF7F0FCEF
:101A60000F4BDA686E682168901B4F1C07D02F68F7
:101A70001B6A9F4209D0964207D8012400E0002447
:101A8000FFF7E8FC2046BDE8F081814205D9081A3D
:101A900020602846FFF7AAFDF1E700202060ECE770
:101AA000140000202DE9FF5F8346DDE90E8799468B
:101AB00016468A469000FFF73BFC05001AD04820E6
:101AC000FFF736FC040012D025630021CDE9024166
:101AD000CDE900874B46324651465846FFF778FA23
:101AE0002046FFF73BF9012004B0BDE8F09F2846EF
:101AF000FFF7BAFC4FF0FF30F6E7000005484169F8
:101B000019B1006B18B10020704701207047022006
:101B100070470000140000200148C06870470000B2
:101B2000140000202DE9F041244C0027206B40B127
:101B3000A069401CA061E06900B101273846BDE8FA
:101B4000F081E668761CE66008D1606BA16B61638A
:101B5000A063206A401C2062FFF74EFBA06A864209
:101B6000E9D3606B006838B1606BC068C5686868AD
:101B7000864204D2A062DEE74FF0FF30FAE7281D6C
:101B8000FFF718FCA86A18B105F11800FFF712FC5E
:101B9000E86A01212269814011432161084900EB73
:101BA000800001EB8000291DFFF73DFCE86A2168F9
:101BB000C96A8842D5D30127D3E70000140000206A
:101BC0008410002070B504004FF000012BD0E06BB2
:101BD000401EE063A36BE26A9A4224D018BB201D2A
:101BE000FFF7E8FB114B124A012150B9E06A00EB04
:101BF000800553F8255025B9156901FA00F0854391
:101C00001561A06BE062C0F10300A061E06A156994
:101C100081402943116100EB800003EB8000211D0E
:101C2000FFF701FC0121084670BD00008410002070
:101C3000140000202DE9F041C068C46804F11800C8
:101C40000746FFF7B7FB144D286B012660B1134818
:101C5000394600BFFFF7E7FBE06A2968C96A884296
:101C600013D90124EE6111E0201DFFF7A3FBE16A07
:101C70002A6906FA01F01043286101EB8100074947
:101C8000643901EB8000211DE4E70024FFF7B4FA7A
:101C90002046BDE8F081000014000020E81000207C
:101CA0002DE9F04700242646FFF7CAFB264D286B96
:101CB000401E2863286BE8BBA968244F0120C9B3E4
:101CC000A7F1640980463868E8B1F868C46804F18F
:101CD0001800FFF76FFB201DFFF76CFBE06A2A6915
:101CE00008FA00F11143296100EB800109EB810042
:101CF000211DFFF798FBE06A2968C96A8842E2D390
:101D0000C5F81C80DFE70CB1FFF776FAAC694CB17F
:101D10004FEA0807FFF706FF00B1EF61641EF9D133
:101D20000020A861E86928B1094901263007086048
:101D300040BF00E003E0BFF34F8FBFF36F8FFFF7AB
:101D400089FB3046BDE8F08714000020E810002031
:101D500004ED00E02DE9F04706461F46154688468B
:101D60002820DDF82090FFF7E3FA04000BD0FFF7FE
:101D70005DF804F11C01C4F81880266081E8A00217
:101D8000201DFFF735FB2046BDE8F0871CB5002479
:101D9000FFF74CF80848006858B107490220091DB0
:101DA000CDE900010023502204A10648FFF77AFE86
:101DB000044620461CBD000050000020546D7220D7
:101DC00053766300A11200002DE9FF41114C1F461C
:101DD0000346266800200A9D002E0ED08DE80E00D6
:101DE00006290FDAFFF78AFE02284FF0000307D01A
:101DF000002269462068FFF703FD04B0BDE8F081CA
:101E00002A46F6E700233A4669463046FFF776FD54
:101E1000F3E7000050000020111213140D0E0F10F4
:101E20000000000100000050481E000000000020DB
:101E3000740000007C080000BC1E0000740000203C
:101E40004C3100008C080000000000000000000081
:101E50000000000000000000000000000000000082
:101E60000000000000000000000000000000000072
:101E70000000000000000000000000000000000062
:101E80000000000000000000000000000000000052
:101E90000000000000000000000000000000000042
:101EA0000000000000000000000000000000000032
:0C1EB00000000000000000000090D003C3
:0400000500000201F4
:00000001FF
